:10000000D0C28CC4E9C2E8C2E7C2E6C2E5C2E4C21B
:10001000E3C2E2C2E1C2E0C2DFC2DEC2DDC2DCC2D4
:10002000DBC2DAC2D9C204030904180372006100FA
:10003000700068006E00650074002E006E006500A0
:1000400074002403470043002F004E0036003400A4
:10005000200074006F0020005500530042002C0067
:100060002000760032001201100100000008401745
:100070007F05010201020001090222000101008046
:100080003209040000010300000009210101000100
:1000900022EC040705810308000A0A03310030003E
:1000A00030003000120101010000000840177F05F8
:1000B00001020102030105010905A10185010901F0
:1000C000A100050175089506150026FF00350046BC
:1000D000FF00093009310933093409350936810235
:1000E00005091500250175019510190129107501E3
:1000F00095108102C0050F0992A1028502099F098E
:10010000A009A409A509A61500250135004501751A
:100110000195058102950375018103099415002558
:10012000013500450175019501810209221501255E
:100130002835014528750795018102C00921A102D2
:1001400085010922150125283501452875089501E5
:1001500091020925A102092609270930093109322E
:100160000933093409400941094209430928250C8A
:1001700015013501450C750895019100C00950091C
:10018000540951150026FF7F350046FF7F66031096
:1001900055FD751095039102550066000009521532
:1001A0000026FF00350046102775089501910209C9
:1001B0005315012508350145087508950191020977
:1001C00055A1020501093009311500250175019578
:1001D000029102C0050F0956950191029505910300
:1001E0000957A1020B01000A000B02000A00661465
:1001F0000055FE150026FF00350047A08C00006664
:1002000000007508950291025500660000C0050FB8
:1002100009A766031055FD150026FF7F350046FF30
:100220007F7510950191026600005500C0050F0909
:100230005AA1028502092215012528350145287594
:100240000895019102095B095D150026FF00350044
:1002500046102795029102095C095E66031055FD60
:1002600026FF7F46FF7F751091024500660000550E
:1002700000C0095FA1028503092215012528350167
:1002800045287508950191020923150025013500BF
:1002900045017504950191020958A1020B01000A5C
:1002A000000B02000A00750295029102C01580251C
:1002B0007F36F0D8461027096075089501910236FF
:1002C000F0D84610270961096295029102150026AF
:1002D000FF003500461027096309647508950291EF
:1002E00002096546102795019102C0096EA1028599
:1002F0000409221501252835014528750895019125
:10030000020970150026FF00350046102775089574
:10031000019102096F1580257F36F0D84610279588
:10032000019102097166140055FE150026FF003583
:100330000047A08C00009102097226FF7F46FF7FD4
:1003400066031055FD751095019102660000550079
:10035000C00973A10285050922150125283501452B
:100360002875089501910209701601FF26FF0036D5
:10037000F0D8461027751095019102C00974A102AA
:10038000850609221501252835014528750895019E
:100390009102097509761580257F36F0D846102719
:1003A000750895029102C00968A102850709221506
:1003B00001252835014528750895019102096C151C
:1003C0000026102735004610277510950191020967
:1003D000691581257F350046FF007508950C92024E
:1003E00001C00966A102850805010930093115819E
:1003F000257F350046FF00750895029102C0050F64
:100400000977A102850A0922150125283501452809
:100410007508950191020978A1020979097A097B89
:1004200015012503750895019100C0097C1500266A
:10043000FF00350046FF009102C00990A102850B24
:1004400009222528150135014528750895019102D5
:10045000C00996A102850C099709980999099A097A
:100460009B099C15012506750895019100C0097D21
:10047000A102850D097E150026FF003500461027D4
:10048000750895019102C0096BA102850E0922151C
:1004900001252835014528750895019102096D153A
:1004A0000026FF00350046FF0075089501910209FE
:1004B0005166031055FD150026FF7F350046FF7F6E
:1004C0007510950191025500660000C009ABA102AC
:1004D00085090925A10209260927093009310932B0
:1004E0000933093409400941094209430928250C07
:1004F00015013501450C75089501B100C0050109CC
:100500003B150026FF01350046FF01750A9501B134
:10051000027506B101C0050F0989A10285020922F1
:10052000252815013501452875089501B102098B6B
:10053000A102098C098D098E25031501350145039A
:1005400075089501B100C009AC150027FFFF000038
:10055000350047FFFF000075109501B100C0097F0D
:10056000A10285030980751095011500350027FF4C
:10057000FF000047FFFF0000B102098326FF00468D
:10058000FF0075089501B10209A909AA7501950234
:100590001500250135004501B10275069501B1032D
:1005A000C0C011241FBECFE5D4E0DEBFCDBF10E038
:1005B000A0E6B0E0E4E4FAE102C005900D92A039B3
:1005C000B107D9F712E0A0E9B0E001C01D92AE304A
:1005D000B107E1F762D434CA13CD85B7826085BF15
:1005E0008BB780648BBF8BE48093E0008AE58093B7
:1005F000DF0008951F93CF93DF936091F000635065
:1006000067FDCFC08091ED00CCE0D0E0C81BD109E0
:10061000CC50DF4F8091EC008D3209F0AEC06830D5
:1006200009F0BDC083EC8093D4008AE5809360001C
:10063000109290008881807621F0CE0115D3AC0114
:1006400084C09A811092DD008981882329F4109258
:10065000DE0042E050E072C0853019F49093F10062
:100660006BC0863009F052C08B81813049F486E638
:1006700090E09093EF008093EE0042E150E042C0A2
:10068000823049F488E790E09093EF008093EE0089
:1006900042E250E037C0833011F58A81882349F463
:1006A00086E290E09093EF008093EE0044E050E00B
:1006B00029C0813049F48AE290E09093EF00809362
:1006C000EE0048E150E01EC08230D1F482E490E0B8
:1006D0009093EF008093EE0044E250E013C081322B
:1006E00049F48AE890E09093EF008093EE0049E0AF
:1006F00050E008C0823221F4CE014AD2AC0102C0DF
:1007000040E050E080E4809390001FC0883029F4DE
:1007100041E050E023EF30E013C0893019F49093AA
:10072000F3000AC08A3019F441E050E007C08B3072
:1007300019F48BE48093E00040E050E02DED30E0D0
:100740003093EF002093EE000DC02FEF4F3F520784
:1007500049F4888187FF02C04E815F8180E88093E1
:10076000900006C08E819F818417950708F4AC0124
:10077000509362004093610012C08091900087FF07
:100780000EC0CE010DD38F3F21F48EE18093600027
:1007900006C0882321F0109262001092610010922E
:1007A000F0008091600084FF60C0809161009091B2
:1007B0006200EFEF8F3F9E0709F457C09C0189301C
:1007C000910510F028E030E0821B930B90936200BB
:1007D000809361008091D40098E889278093D400A9
:1007E000122F222391F16091EE007091EF00809121
:1007F000900086FF13C09B01C5EDD0E01150412F42
:1008000050E01F5FDA01AA52BF4FF901849189932A
:100810002F5F3F4FCA17DB07C1F70FC0DB01E5EDC4
:10082000F0E01150412F50E01F5F9A012A523F4FD4
:100830008D918193E217F307D9F7CA010196860FCC
:10084000971F9093EF008093EE0085ED90E0612F6D
:1008500061D0612F6C5F6C3031F08FEF9FEF909320
:100860006200809361006093600094E180B38570C2
:1008700031F49150D9F71092F1001092EB00DF9112
:10088000CF911F9108951F93DC01162F8091DF00F7
:1008900084FF07C08091E00098E889278093E000FA
:1008A00003C08AE58093DF00912FE1EEF0E08D91A7
:1008B000819391501916DCF381EE90E0612F2AD0DC
:1008C0001C5F1093DF001F910895A82FB92F8FEFA1
:1008D0009FEF1BC02D918227282F22952827722F4A
:1008E000269526952727239526952170782F892FE1
:1008F00082272195207C922F22277695279597276E
:1009000082277695279597278227615018F780953B
:1009100090950895DADF8D939D930895CF93CFB787
:10092000CF93C395809BE9F7809B09C0809B07C04C
:10093000809B05C0809B03C0809B01C0A3C0DF9348
:10094000C091ED00DD27CC50DF4F809B02C0DF91CE
:10095000EBCF2F930F931F9300B32FEF00FB20F9E2
:100960004F933F9310B34FEF012700FB21F93BE07A
:1009700031C04E7F012F10B3216028C0102F4D7F52
:100980002260000000B329C04B7F2460012F0000CB
:1009900010B32BC010B3477F28602AC04F7E00B32E
:1009A00020612CC04F7D10B320622FC04F7B00B35D
:1009B000206432C0422700B349934FEF0000102754
:1009C00010FB20F910B31570C9F1297F91F20127AE
:1009D00000FB21F900B3237F89F2315058F1102731
:1009E00010FB22F910B3277E79F2012700FB23F9CF
:1009F0002F7C81F200B3102710FB24F92F7971F2BC
:100A000000C010B3012700FB25F92F7359F200C075
:100A100000B3102710FB26F9223040F200C010B3BB
:100A2000012700FB27F9243028F64F77206810B300
:100A30000000F9CF10E41ABF002719C03B503195D0
:100A4000C31BD04010E41ABF0881033CF9F00B34FB
:100A5000E9F02091EB001981110F1213EDCF4A81BB
:100A6000441F093641F10D3211F0013E29F7009380
:100A7000F2003F914F911F910F912F91DF91CAB7D3
:100A8000C6FD4FCFCF91CFBFCF9118952091F200E7
:100A9000222379F31091F000112369F534306AF1C3
:100AA0003093F0002093EC001091ED003BE0311BFF
:100AB0003093ED0022C00091F0000130E4F40AE52B
:100AC0004F7049F43091600034FD19C0009360000C
:100AD000C4EDD0E018C03091DF0034FD10C00093A9
:100AE000DF00C0EED0E00FC02795A8F45150A9F464
:100AF000220F0000F9CF4AE503C042ED01C0432FA9
:100B0000C4E1D0E032E011B31560909A11BB02B39A
:100B100020E415E05F93012756E002BB279520F4FF
:100B2000515021F4220FF9CF012756E000003B5A23
:100B300002BBD0F2279528F4515029F4220F00006F
:100B4000F9CF012756E0279502BB20F4515021F43C
:100B5000220FF9CF012756E02991332302BB21F65A
:100B60000A7F1091F100110FC651D04002BB11F065
:100B70001093EB0010E41ABF016011B31A7F402FED
:100B80004A7F5F9100C000C002BB11BB42BB71CF66
:100B9000FC018081807619F58181863001F58381A1
:100BA000813019F08232D9F40DC080919500909176
:100BB00096009093EF008093EE0080919700282F8D
:100BC00030E00FC080919100909192009093EF00DF
:100BD0008093EE00209193003091940002C020E0B9
:100BE00030E0C9010895E0919800F09199003097A4
:100BF00049F00288F389E02D309721F0992787FD8D
:100C0000909509950895DC01E0919800F091990084
:100C1000309719F56130710519F020E030E022C0FD
:100C200081E08C938FE711968C93119712968C9399
:100C3000129713968C93139714968C93149715967A
:100C40008C93159716968C93169717961C92179758
:100C500018961C9229E030E005C00088F189E02D4B
:100C600009959C01C9010895DC014DE950E05093BC
:100C7000EF004093EE008C918076803209F071C0D5
:100C800011962C911197223009F440C0233020F4A2
:100C9000213009F066C007C0293009F45FC02A304E
:100CA00009F05FC044C013968C911397813021F0F6
:100CB000833009F053C00AC012966C91662309F480
:100CC0004DC0CA0170E09FDF9C014DC012966C912F
:100CD000623061F460939D0020939E0020939F00FA
:100CE0008AE08093A0008093A1000DC06330B1F52D
:100CF00060939D0020939E0020939F008FEF809330
:100D0000A0002093A10025E030E02DC012966C9148
:100D1000862F8150823028F5862F90E08A559F4F8C
:100D20009093EF008093EE0021E030E01CC012961B
:100D3000EC911297EE2339F413968C918093A700CF
:100D40008093A8000EC08E2F8150823050F4F0E0C6
:100D5000EA55FF4F13968C91808303C02FEF3FEF2E
:100D600002C020E030E0C90108958091AA0090916E
:100D7000AB00892B11F410929A0080919A0088237D
:100D800011F431DF089580919B0087FF02C081E05C
:100D90002ADF80919C0087FF02C081E024DF089554
:100DA000FC01662309F448C08081853089F08630D3
:100DB00030F4813049F0843009F03EC010C08930F1
:100DC00019F08A30C9F50FC081818093A90034C021
:100DD0008181813089F5828180939B002CC0828142
:100DE00080939C0028C0643039F5838190E023E033
:100DF000880F991F2A95E1F79093AB008093AA0082
:100E0000818190E08F7790708130910531F0813051
:100E1000910594F00397029778F48281823029F04B
:100E2000833039F0813041F401C081E080939A0031
:100E300002C010929A0099DF81E008950F931F93EA
:100E4000CF93DF93BC018091DF0084FF21C08DE947
:100E500090E0D9DEC0E0D0E0082F112707FD109503
:100E600014C0CE0183569F4FB8016C1B7D0B6930B7
:100E7000710514F068E070E006DD02C0BBDBA895E8
:100E80008091DF0084FFFACF2896C017D1074CF37A
:100E9000DF91CF911F910F9108952F923F924F9222
:100EA0005F926F927F928F929F92AF92BF92CF92FA
:100EB000DF92EF92FF920F931F93DF93CF9300D0B7
:100EC000CDB7DEB71A82198214BABB24BA94B5BA68
:100ED000E8EFCE2EC2BA15E011BB78EEE72E70E82F
:100EE000F72EC7010197F1F711BA13BF0FE005BD47
:100EF00064ECD62ED3BC86EB90E090939200809366
:100F000091009BD4909394008093930084EA90E0A6
:100F100090939600809395004FD18093970014BAD8
:100F2000B5BAC2BA11BBC7010197F1F711BA13BF25
:100F300005BDD3BC85D488E190E00FB6F894A895A0
:100F400081BD0FBE01BD49DB7894BB24AA24A394C4
:100F5000EE24FF24222423942E010894411C511CCA
:100F600051E0652E712C40E8342E3CE2832E31E0B6
:100F7000932E04C0BB2402C0EE24FF24A8952FE1C9
:100F8000E216F10424F010929900109298008091DA
:100F9000980090919900892B09F05CC080E023DED5
:100FA00029DB81E090E04ADF8CE291E0F4013197A7
:100FB000F1F70197D9F71EDBF4D48230910539F0AF
:100FC0008330910589F00197B9F62AD401C078D20F
:100FD000FC0190939900809398000284F385E02DA2
:100FE000099580E000DEC8CF6BD2FC019093990098
:100FF000809398000284F385E02D0995E091980094
:10100000F09199000488F589E02D09958823F1F481
:10101000F1DA80E991E0F4013197F1F70197D9F71E
:10102000E9DAFED3FC019093990080939800028442
:10103000F385E02D0995E0919800F09199000488DE
:10104000F589E02D0995882309F496CF80E0CBDD62
:10105000EE24FF24A895CEDAAA2099F086DEE0914E
:101060009800F09199000484F585E02D0995882376
:1010700021F4AA24EE24FF2404C00894E11CF11CEE
:10108000AA2408B607FE3EC038BEBB2009F03AC00D
:101090006CDE85B7806885BF889585B78F7785BFFB
:1010A000C4010197F1F7E0919800F0919900048450
:1010B000F585E02D0995882319F4EE24FF2403C05B
:1010C0000894E11CF11C00E010E013C068010894D2
:1010D000C11CD11C0684F785E02DC6010995882323
:1010E00039F0C30102C0880F991F0A95E2F7B82AA8
:1010F0008601E0919800F09199008481958108170C
:10110000190724F308B600FE35C028BE8091AA0056
:101110009091AB00009749F02FEF8F3F920729F095
:1011200001979093AB008093AA00E0919800F09112
:10113000990044815581D20120E030E018C0F901C6
:10114000E955FF4FE081EE2379F08C91853018F05E
:1011500085508C9309C0EC93C301022E02C0880F06
:10116000991F0A94E2F7B82A2F5F3F4F1196241770
:1011700035072CF3BB2009F401CF00E010E0CB2CA5
:10118000DD24C7FCD0940EC0C601002E02C0959588
:1011900087950A94E2F780FF03C0C80101964EDEEE
:1011A0000F5F1F4FE0919800F09199008481958125
:1011B000081719074CF3DECE82E190E00895909372
:1011C000AD008093AC000895009741F0DC01E0EBA6
:1011D000F0E089E001900D928150E1F7A9EBB0E0D9
:1011E000E0EBF0E089E001900D928150E1F789E0B9
:1011F00090E0089580EB90E069EB70E049E050E00A
:101200000BD408950F931F93DF93CF93CDB7DEB721
:1012100029970FB6F894DEBF0FBECDBF1982CE015D
:10122000019661E070E011D3883109F01FC180E4BC
:101230008A8383E08B831C828091AC009091AD0007
:10124000892B11F081E08C838E010E5F1F4FC80146
:1012500063E070E0FAD2803409F008C188E0F80158
:1012600011928A95E9F74A8120E030E060E870E069
:10127000F901E65EFE4F8081882339F0CB01022E12
:1012800002C0959587950A94E2F7482B2F5F3F4F50
:101290002830310569F74A834B8120E030E060E86F
:1012A00070E0F901EE5DFE4F8081882339F0CB01BB
:1012B000022E02C0959587950A94E2F7482B2F5F7E
:1012C0003F4F2830310569F740954B834C8120E032
:1012D00030E060E870E0F901E65DFE4F8081882330
:1012E00039F0CB01022E02C0959587950A94E2F75A
:1012F000482B2F5F3F4F2830310569F74C834D81D4
:1013000020E030E060E870E0F901EE5CFE4F8081A3
:10131000882311F080E007C0CB01022E02C0959512
:1013200087950A94E2F7482B2F5F3F4F283031050D
:1013300059F74D834E8120E030E060E870E0F9011C
:10134000E65CFE4F8081882339F0CB01022E02C07B
:10135000959587950A94E2F7482B2F5F3F4F2830E9
:10136000310569F740954E834F8120E030E060E819
:1013700070E0F901EE5BFE4F8081882339F0CB01EC
:10138000022E02C0959587950A94E2F7482B2F5FAD
:101390003F4F2830310569F740954F83488520E05D
:1013A00030E061E070E0F901E35FFE4F8081882367
:1013B00039F0CB01022E02C0880F991F0A94E2F780
:1013C000482B2F5F3F4F2530310569F720E030E093
:1013D00060E270E0F901ED5EFE4F8081882339F014
:1013E000CB01022E02C0880F991F0A94E2F7482B06
:1013F0002F5F3F4F2330310569F74887498520E04B
:1014000030E061E070E0F901EA5EFE4F8081882300
:1014100039F0CB01022E02C0880F991F0A94E2F71F
:10142000482B2F5F3F4F2430310569F7498781E012
:101430008093B000A1EBB0E0FE01329686E001900F
:101440000D928150E1F78091AE009091AF00892B11
:1014500029F08FE78093B5008093B600888580934C
:10146000B70089858093B80080E001C081E02996AB
:101470000FB6F894DEBF0FBECDBFCF91DF911F91A5
:101480000F910895BFDE90E0882309F491E0892F41
:101490000895B8DE882399F480911301882359F0C8
:1014A00080911401882339F081E090E09093AF009F
:1014B0008093AE0008951092AF001092AE00089590
:1014C00086EB90E09093660080936500B6D1E5E6E8
:1014D000F0E092938293CF01089520918F00253000
:1014E00079F0222369F0892B31F0233049F082E032
:1014F00080938F000895213019F084E080938F004D
:101500000895CF92DF92EF92FF921F93DF93CF93D4
:101510000F92CDB7DEB785E080938F0010E08CE2AC
:10152000C82E81E0D82E7E010894E11CF11C62D8FF
:101530008CE291E0F6013197F1F70197D9F7198222
:10154000C70161E070E081D1489711F481E004C0E7
:101550001F5F1F3061F780E00F90CF91DF911F91E7
:10156000FF90EF90DF90CF900895009741F0DC015D
:10157000E2ECF0E089E001900D928150E1F7ABECF4
:10158000B0E0E2ECF0E089E001900D928150E1F7EB
:1015900089E090E0089582EC90E06BEC70E049E027
:1015A00050E03AD208951F93DF93CF93CDB7DEB7C3
:1015B000A6970FB6F894DEBF0FBECDBF1982CE013D
:1015C000019661E070E041D1883119F010928F00EE
:1015D00067C080912101882331F080918F00853090
:1015E00011F410928F0080912101882319F485E075
:1015F00080938F0080918F008230D9F0843081F108
:10160000882309F044C083E0898380E88A8381E0ED
:101610008B83CE01049660E870E042E250E009D28C
:10162000CE01019663E270E010D1882381F184E05D
:101630002CC013E0198380EC8A838BE18B83CE016D
:10164000049661E070E040E250E0F3D1CE010196F3
:1016500063E270E0FAD08823D1F010938F0017C0B6
:1016600083E0898380EC8A838BE18B8380E2FE01B7
:101670003496DF011D928A95E9F7CE01019663E267
:1016800070E0E3D0882319F081E080938F0081E03F
:101690008983CE01019661E070E0D7D0803211F0ED
:1016A0008FEFB0C019821A821B821C8240E020E0BA
:1016B00030E061E070E0F901E65FFE4F8081882351
:1016C00039F0CB01022E02C0880F991F0A94E2F76D
:1016D000482B2F5F3F4F2430310569F720E030E081
:1016E00060E170E0F901EA5EFE4F8081882339F005
:1016F000CB01022E02C0880F991F0A94E2F7482BF3
:101700002F5F3F4F2430310569F74B8380911401DF
:1017100020E0811121E09C81922B809115018111A3
:1017200082E0892B8C83498120E030E060E870E022
:10173000F901E65EFE4F8081882339F0CB01022E4D
:1017400002C0959587950A94E2F7482B2F5F3F4F8B
:101750002830310569F749834A8120E030E060E8AC
:1017600070E0F901EE5DFE4F8081882339F0CB01F6
:10177000022E02C0959587950A94E2F7482B2F5FB9
:101780003F4F2830310569F74A8381E08093C200DA
:10179000898181588093C3008FE7982F941B909381
:1017A000C4008093C5008093C6008093C7008093D7
:1017B000C8008B818093C9009C819093CA0080915E
:1017C0000E01882319F094609093CA0080910F0154
:1017D000882329F08091CA0088608093CA00809194
:1017E0001001882329F08091CA0080618093CA008B
:1017F00080911101882331F08091CA00806280932A
:10180000CA0080E0A6960FB6F894DEBF0FBECDBF2B
:10181000CF91DF911F910895A09AA898C4DE0895F2
:1018200086EB90E090937C0080937B0006D0EBE702
:10183000F0E092938293CF0108958CEE94E00895A6
:10184000A598AD98BC9AC4980895EF92FF920F9313
:101850001F93CF93DF937C01662309F44FC070E0A0
:1018600020E030E0E0E0F0E011C088818423FD0159
:10187000E65FFE4F808311964695A017B107A9F742
:101880002F5F3F4F2617370754F4FD01DF0140E873
:10189000E701C20FD31F8F01085F1F4FE6CFEAE0B9
:1018A000F1E0CF93DF93EF93FF930191002311F0C9
:1018B00049F416C00000A59A19E00FD0A598119719
:1018C000A1F70EC0A59A11E008D0A59815E005D0A3
:1018D00000000000119749F703C01A95F1F7089529
:1018E0000000FF91EF91DF91CF91A59A11E0F5DF14
:1018F000A5980FEF0A9511F09D9BFCCFEAE0F1E06F
:10190000EF93FF93112700270395A1F09D99FCCF3A
:1019100008C004E6039572F09D99FCCF139551F031
:10192000019304E6039532F09D9BFCCF139511F0D3
:101930000193EFCFFF91EF91612F70E06115710579
:1019400031F110FF24C040E050E020E030E00CC056
:101950008081F901E75FFE4F9081E0E0891708F48C
:10196000E1E0EC934F5F5F4FDA01A65FBE4FF901F4
:10197000E65FFE4F2E5F3F4F411750F384E18A959B
:10198000F1F79B01215030403595279502C020E0AA
:1019900030E0C901DF91CF911F910F91FF90EF903F
:1019A0000895DF93CF930F92CDB7DEB71982CE01A2
:1019B000019661E070E049DF009719F420E030E023
:1019C00026C0489711F580910E01882311F098E008
:1019D00001C090E080910F0181119460809110010D
:1019E0008111926080911101811191609A3028F4E7
:1019F000983028F4953049F405C09B3031F422E04A
:101A000030E005C021E030E002C023E030E0C90151
:101A10000F90CF91DF910895FB01DC0104C08D91FF
:101A20000190801921F441505040C8F7881B990B50
:101A30000895DC0101C06D9341505040E0F70895D6
:041A4000F894FFCF48
:101A44005AFFFF00000000010000000000490A02E4
:101A540009FA08E408DF08420A0000000001000057
:101A64000000000C0CD30ACB0AB50A6D0A810A05E2
:00000001FF
